:1000000019C02BC02AC029C028C027C026C025C0BF
:1000100024C023C022C021C020C01FC01EC01DC0DC
:100020001CC01BC01AC019C018C017C016C015C00C
:1000300014C013C011241FBECFEFD2E0DEBFCDBF6E
:1000400011E0A0E0B1E0E2EDF0E002C005900D9219
:10005000AA30B107D9F702D03AC0D2CF84B18963B0
:1000600084B98AB18FEF8AB9289A20E033E045B18C
:10007000822F632F20D0E92FF0E0E050FF4F8081E6
:10008000842B85B99BB1A22FB0E0AD5FBE4F8C91A0
:10009000892B8BB987EA91E60197F1F700C0000040
:1000A00095B180818095892385B91BB82F5F263053
:1000B000F0F220E0DCCF991B79E004C0991F96177D
:1000C00008F0961B881F7A95C9F780950895F894D3
:0200D000FFCF60
:0A00D200091121120624210918006B
:00000001FF
